:1000000019C033C032C031C064C12FC02EC02DC052
:100010002CC02BC02AC029C028C0E4C126C025C0DE
:1000200024C023C022C021C020C01FC01EC01DC0CC
:100030001CC01BC011241FBECFEFD4E0DEBFCDBF5C
:1000400011E0A0E0B1E0E0E9FAE002C005900D9215
:10005000A033B107D9F721E0A0E3B1E001C01D92C0
:10006000AB36B207E1F7F6D111C5CACF83E306C0BC
:10007000E7E8F3E13197F1F700C000008150C1F7E4
:100080000895419A8DE08A95F1F70000419808950E
:1000900095B1869586958C73937C892B85B9F1CF24
:1000A000CF93C82F662311F0409A01C040988C2F3F
:1000B000EFDF8C2F8295807FEBDF8BE004C095E82B
:1000C0009A95F1F700008150D1F7CF91089560E043
:1000D000E7CF61E0E5CFCF93DF93EC0101C0F9DF1B
:1000E00089918111FCCFDF91CF910895D1DF8FE409
:1000F00093EC0197F1F700C000000895B7DF80E3AB
:10010000F5DF80E3F3DF80E3F1DF80E2EFDF88E219
:10011000DEDF8CE0DCDF81E0DADFA8DF80E8D7DF3C
:100120008EE191E0D8DF80ECD2DF8DE091E0D3CF9B
:10013000CF92DF92EF92FF920F931F93CF93DF93B3
:100140007B018C01E42FFF27E7FDF095E050FF4F86
:100150008081BDDF20E030E44CE156E46E2D7F2D40
:10016000802F912F2CD487FD0FC020E030E543EC89
:1001700057E46E2D7F2D802F912FD2D287FF04C0A0
:1001800080E2A7DFC7E301C0C0E020E030E543EC38
:1001900057E46E2D7F2D802F912F11D487FF02C041
:1001A000D5E002C0D6E0C7E320E034E244E759E4FA
:1001B0006E2D7F2D802F912F02D487FD02C0DF5F2F
:1001C000C7E320E030E040E85FE36E2D7F2D802F15
:1001D000912FF5D387FF0DC071C02DEC3CEC4CEC9A
:1001E0005DE36E2D7F2D802F912FEDD37B018C0150
:1001F000CF5F20E030E040E251E46E2D7F2D802F74
:10020000912FDDD387FFE9CF27E137EB41E558E3B5
:100210006E2D7F2D802F912F1FD2D62EF72E8C0181
:1002200020E030E040E251E4912FC9D387FD0DC0BA
:100230002DEC3CEC4CEC5DE36D2D7F2D802F912F50
:10024000C2D3D62EF72E8C01CF5FE12C6D2D7F2DE2
:10025000802F912FD1D2C62E862F805D3ADFEC12EF
:1002600002C08EE236DF6C2D772767FD7095872FF1
:10027000972FF5D29B01AC016D2D7F2D802F912FF3
:10028000EAD120E030E040E251E49DD3D62EF72EB3
:100290008C01E39485E0E812D9CFC5E003C080E388
:1002A00018DFCF5FCD17DCF380E2DF91CF911F9194
:1002B0000F91FF90EF90DF90CF900BCF84E091E013
:1002C000DF91CF911F910F91FF90EF90DF90CF9032
:1002D00002CF1F920F920FB60F9211242F933F93CC
:1002E0004F938F939F93AF93BF9386B180958C73F9
:1002F000409130014095482380933001442309F414
:1003000065C02091840030918500809161019091B9
:100310006201B09B02C037FF0196A0E0B0E0DC01B3
:1003200099278827820F931FA11DB11D42FF12C07C
:1003300020915101309152012F5F3F4F3093520174
:10034000209351018093410190934201A093430176
:10035000B093440143FF12C02091530130915401E6
:100360002F5F3F4F309354012093530180934501F9
:1003700090934601A0934701B093480144FF12C0F7
:1003800020915501309156012F5F3F4F3093560118
:10039000209355018093490190934A01A0934B010A
:1003A000B0934C01407291F0209157013091580167
:1003B0002F5F3F4F309358012093570180934D0199
:1003C00090934E01A0934F01B0935001BF91AF9114
:1003D0009F918F914F913F912F910F900FBE0F9052
:1003E0001F9018951F920F920FB60F9211248F93A2
:1003F0009F93EF93FF938091610190916201019629
:1004000090936201809361017894E3E6F1E080814A
:100410009181019691838083E5E6F1E0808191816D
:10042000019691838083E7E6F1E0808191810196D6
:1004300091838083E9E6F1E0808191810196918347
:100440008083FF91EF919F918F910F900FBE0F903E
:100450001F901895CF93DF93CDB7DEB727970FB6D0
:10046000F894DEBF0FBECDBF80E88093610010928C
:1004700061009CE398B983E085B92FEF2BB994B95B
:1004800087B93CDE04E610E0F1DD01501109E1F727
:100490008E010F5F1F4F70E0E72E71E0F72E6E01A7
:1004A00025E0C20ED11CF80111928F01F701819154
:1004B0007F010DDE84E091E00EDE0C151D0599F73D
:1004C00081E08093810080936F008CE380936C00C7
:1004D00082E0809368007894F4E0FD832D812F5FA3
:1004E0002D8324300CF01D8280916F008E7F8093CD
:1004F0006F003D81032F112707FD10959801220FF2
:10050000331FF901ED59FE4F80819181F901EF5AB6
:10051000FE4F20803180A801440F551F440F551F06
:100520005F834E83FA01EF5BFE4FC080D180E28093
:10053000F38040916F00416040936F0084369105D5
:1005400068F2F901E75AFE4F20813181B101621B47
:10055000730BEE81FF81EF5CFE4F80809180A28063
:10056000B3806115710509F451C0A70196012819DE
:1005700039094A095B0949015A0130E483163BE411
:1005800093063CE4A306B10408F440C0E1E0F0E0C7
:10059000EC0FFD1FE00FF11F80818823C9F080E080
:1005A00090E05BD120E836E948E95BE40CD22B010E
:1005B0003C01C501B40151D19B01AC01C301B201A1
:1005C000B3D020E030E040E752E4FDD14D81B0DD12
:1005D000E1E0F0E0EC0FFD1FE00FF11F41E0408390
:1005E000000F111FF801E75AFE4F31822082EE8181
:1005F000FF81EF5CFE4FC082D182E282F382809164
:100600006F008E7F80936F00F8011BC088359D447A
:1006100008F464CFF801E050FF4F808158DD84E09A
:1006200091E059DDE1E0F0E0EC0FFD1FE00FF11F7C
:10063000108280916F008E7F80936F00F801EE0F23
:10064000FF1FED59FE4F1182108280916F00816073
:1006500080936F0043CF5058BB27AA270ED075C197
:1006600066D130F06BD120F031F49F3F11F41EF4CD
:100670005BC10EF4E095E7FB51C1E92F77D180F320
:10068000BA17620773078407950718F071F49EF58F
:100690008FC10EF4E0950B2EBA2FA02D0B01B901DE
:1006A00090010C01CA01A0011124FF27591B99F0E8
:1006B000593F50F4503E68F11A16F040A22F232FF4
:1006C000342F4427585FF3CF469537952795A79544
:1006D000F0405395C9F77EF41F16BA0B620B730BEB
:1006E000840BBAF09150A1F0FF0FBB1F661F771F5C
:1006F000881FC2F70EC0BA0F621F731F841F48F411
:10070000879577956795B795F7959E3F08F0B3CF96
:100710009395880F08F09927EE0F97958795089580
:10072000D9D008F481E008950CD00FC107D140F072
:10073000FED030F021F45F3F19F0F0C0511139C103
:10074000F3C014D198F39923C9F35523B1F3951B42
:10075000550BBB27AA2762177307840738F09F5FE2
:100760005F4F220F331F441FAA1FA9F333D00E2E51
:100770003AF0E0E830D091505040E695001CCAF7BE
:1007800029D0FE2F27D0660F771F881FBB1F261783
:1007900037074807AB07B0E809F0BB0B802DBF0156
:1007A000FF2793585F4F2AF09E3F510568F0B6C06F
:1007B00000C15F3FECF3983EDCF386957795679533
:1007C000B795F7959F5FC9F7880F911D9695879507
:1007D00097F90895E1E0660F771F881FBB1F621726
:1007E00073078407BA0720F0621B730B840BBA0BE4
:1007F000EE1F88F7E095089504D06894B111D9C030
:100800000895BCD088F09F5790F0B92F9927B75121
:10081000A0F0D1F0660F771F881F991F1AF0BA95C4
:10082000C9F712C0B13081F0C3D0B1E00895C0C0A3
:10083000672F782F8827B85F39F0B93FCCF38695BA
:1008400077956795B395D9F73EF490958095709517
:1008500061957F4F8F4F9F4F0895E89409C097FB94
:100860003EF490958095709561957F4F8F4F9F4F87
:100870009923A9F0F92F96E9BB279395F6958795CB
:1008800077956795B795F111F8CFFAF4BB0F11F48E
:1008900060FF1BC06F5F7F4F8F4F9F4F16C0882335
:1008A00011F096E911C0772321F09EE8872F762F6B
:1008B00005C0662371F096E8862F70E060E02AF0AC
:1008C0009A95660F771F881FDAF7880F9695879598
:1008D00097F90895990F0008550FAA0BE0E8FEEF6D
:1008E00016161706E807F907C0F012161306E407F4
:1008F000F50798F0621B730B840B950B39F40A26ED
:1009000061F0232B242B252B21F408950A2609F4CA
:10091000A140A6958FEF811D811D089597F99F67CE
:1009200080E870E060E008959FEF80EC0895002477
:100930000A941616170618060906089500240A9444
:1009400012161306140605060895092E0394000CCA
:1009500011F4882352F0BB0F40F4BF2B11F460FF59
:1009600004C06F5F7F4F8F4F9F4F089557FD905882
:10097000440F551F59F05F3F71F04795880F97FB63
:10098000991F61F09F3F79F087950895121613061D
:100990001406551FF2CF4695F1DF08C0161617064C
:1009A0001806991FF1CF8695710561050894089581
:1009B000E894BB2766277727CB0197F908958ADF4C
:1009C00008F48FEF08950BD0C0CFB1DF28F0B6DF69
:1009D00018F0952309F0A2CFA7CF1124EACFC6DFE4
:1009E000A0F3959FD1F3950F50E0551F629FF00142
:1009F000729FBB27F00DB11D639FAA27F00DB11D9B
:100A0000AA1F649F6627B00DA11D661F829F222723
:100A1000B00DA11D621F739FB00DA11D621F839FAA
:100A2000A00D611D221F749F3327A00D611D231F80
:100A3000849F600D211D822F762F6A2F11249F57CE
:100A400050408AF0E1F088234AF0EE0FFF1FBB1FF1
:100A5000661F771F881F91505040A9F79E3F510590
:100A600070F05CCFA6CF5F3FECF3983EDCF3869549
:100A700077956795B795F795E7959F5FC1F7FE2B3B
:100A8000880F911D9695879597F90895F894FFCF53
:100A90008189C1C92020202D2E2D20200020332E19
:100AA0004B616E616C20342E4B616E616C002031A5
:100AB0002E4B616E616C20322E4B616E616C0000BA
:00000001FF
